 FARCmds

 Timestamp is 559d99f8 (Thu Jul 09 00:45:28 2015)

 Preferred load address is 10000000

 Start         Length     Name                   Class
 0001:00000000 000000e0H .idata$5                CODE
 0001:000000e0 000004dcH .rdata                  CODE
 0001:000005c0 00004e34H .text                   CODE
 0001:000053f4 00000064H .idata$2                CODE
 0001:00005458 00000014H .idata$3                CODE
 0001:0000546c 000000e0H .idata$4                CODE
 0001:0000554c 000003d8H .idata$6                CODE
 0001:00005930 000000a5H .edata                  CODE
 0002:00000000 000000acH .data                   DATA
 0002:000000b0 000015b8H .bss                    DATA
 0003:00000000 00000058H .rsrc$01                DATA
 0003:00000060 00000378H .rsrc$02                DATA

  Address         Publics by Value              Rva+Base       Lib:Object

 0000:00000000       ___safe_se_handler_table   00000000     <absolute>
 0000:00000000       ___safe_se_handler_count   00000000     <absolute>
 0001:00000000       __imp__RegCloseKey@4       10001000     advapi32:ADVAPI32.dll
 0001:00000004       __imp__RegQueryValueExW@24 10001004     advapi32:ADVAPI32.dll
 0001:00000008       __imp__RegOpenKeyExW@20    10001008     advapi32:ADVAPI32.dll
 0001:0000000c       __imp__IsTextUnicode@12    1000100c     advapi32:ADVAPI32.dll
 0001:00000010       \177ADVAPI32_NULL_THUNK_DATA 10001010     advapi32:ADVAPI32.dll
 0001:00000014       __imp__GetConsoleAliasesW@12 10001014     kernel32:KERNEL32.dll
 0001:00000018       __imp__GetConsoleAliasesLengthW@4 10001018     kernel32:KERNEL32.dll
 0001:0000001c       __imp__lstrcatW@8          1000101c     kernel32:KERNEL32.dll
 0001:00000020       __imp__GetLastError@0      10001020     kernel32:KERNEL32.dll
 0001:00000024       __imp__GetModuleFileNameW@12 10001024     kernel32:KERNEL32.dll
 0001:00000028       __imp__CloseHandle@4       10001028     kernel32:KERNEL32.dll
 0001:0000002c       __imp__ReadFile@20         1000102c     kernel32:KERNEL32.dll
 0001:00000030       __imp__CreateFileW@28      10001030     kernel32:KERNEL32.dll
 0001:00000034       __imp__MultiByteToWideChar@24 10001034     kernel32:KERNEL32.dll
 0001:00000038       __imp__GetACP@0            10001038     kernel32:KERNEL32.dll
 0001:0000003c       __imp__GetConsoleOutputCP@0 1000103c     kernel32:KERNEL32.dll
 0001:00000040       __imp__SetConsoleTitleW@4  10001040     kernel32:KERNEL32.dll
 0001:00000044       __imp__GetConsoleWindow@0  10001044     kernel32:KERNEL32.dll
 0001:00000048       __imp__GetCurrentDirectoryW@8 10001048     kernel32:KERNEL32.dll
 0001:0000004c       __imp__RemoveDirectoryW@4  1000104c     kernel32:KERNEL32.dll
 0001:00000050       __imp__DeleteFileW@4       10001050     kernel32:KERNEL32.dll
 0001:00000054       __imp__GetFileSize@8       10001054     kernel32:KERNEL32.dll
 0001:00000058       __imp__WriteConsoleW@20    10001058     kernel32:KERNEL32.dll
 0001:0000005c       __imp__ExpandEnvironmentStringsW@12 1000105c     kernel32:KERNEL32.dll
 0001:00000060       __imp__GetTempFileNameW@16 10001060     kernel32:KERNEL32.dll
 0001:00000064       __imp__CreateDirectoryW@8  10001064     kernel32:KERNEL32.dll
 0001:00000068       __imp__SearchPathW@24      10001068     kernel32:KERNEL32.dll
 0001:0000006c       __imp__GetEnvironmentVariableW@12 1000106c     kernel32:KERNEL32.dll
 0001:00000070       __imp__WaitForSingleObject@8 10001070     kernel32:KERNEL32.dll
 0001:00000074       __imp__CreateThread@24     10001074     kernel32:KERNEL32.dll
 0001:00000078       __imp__CreateProcessW@40   10001078     kernel32:KERNEL32.dll
 0001:0000007c       __imp__SetCurrentDirectoryW@4 1000107c     kernel32:KERNEL32.dll
 0001:00000080       __imp__SetConsoleCursorPosition@8 10001080     kernel32:KERNEL32.dll
 0001:00000084       __imp__GetConsoleScreenBufferInfo@8 10001084     kernel32:KERNEL32.dll
 0001:00000088       __imp__SetConsoleMode@8    10001088     kernel32:KERNEL32.dll
 0001:0000008c       __imp__GetConsoleMode@8    1000108c     kernel32:KERNEL32.dll
 0001:00000090       __imp__GetStdHandle@4      10001090     kernel32:KERNEL32.dll
 0001:00000094       __imp__HeapFree@12         10001094     kernel32:KERNEL32.dll
 0001:00000098       __imp__GetProcessHeap@0    10001098     kernel32:KERNEL32.dll
 0001:0000009c       __imp__HeapAlloc@12        1000109c     kernel32:KERNEL32.dll
 0001:000000a0       __imp__HeapReAlloc@16      100010a0     kernel32:KERNEL32.dll
 0001:000000a4       __imp__GetFileAttributesW@4 100010a4     kernel32:KERNEL32.dll
 0001:000000a8       __imp__lstrlenW@4          100010a8     kernel32:KERNEL32.dll
 0001:000000ac       __imp__lstrcpyW@8          100010ac     kernel32:KERNEL32.dll
 0001:000000b0       __imp__Sleep@4             100010b0     kernel32:KERNEL32.dll
 0001:000000b4       __imp__lstrcpynW@12        100010b4     kernel32:KERNEL32.dll
 0001:000000b8       \177KERNEL32_NULL_THUNK_DATA 100010b8     kernel32:KERNEL32.dll
 0001:000000bc       __imp__UuidFromStringW@8   100010bc     rpcrt4:RPCRT4.dll
 0001:000000c0       \177RPCRT4_NULL_THUNK_DATA 100010c0     rpcrt4:RPCRT4.dll
 0001:000000c4       __imp__GetWindowTextW@12   100010c4     user32:USER32.dll
 0001:000000c8       __imp__GetWindowTextLengthW@4 100010c8     user32:USER32.dll
 0001:000000cc       \177USER32_NULL_THUNK_DATA 100010cc     user32:USER32.dll
 0001:000000d0       __imp__CoUninitialize@0    100010d0     ole32:ole32.dll
 0001:000000d4       __imp__CoCreateInstance@20 100010d4     ole32:ole32.dll
 0001:000000d8       __imp__CoInitialize@4      100010d8     ole32:ole32.dll
 0001:000000dc       \177ole32_NULL_THUNK_DATA  100010dc     ole32:ole32.dll
 0001:000000e0       ??_C@_1BE@KBOCGMKN@?$AAS?$AAe?$AAp?$AAa?$AAr?$AAa?$AAt?$AAo?$AAr?$AA?$AA@ 100010e0     FARCmds.obj
 0001:000000f4       ??_C@_1BI@BKNCFIOG@?$AAM?$AAa?$AAx?$AAD?$AAa?$AAt?$AAa?$AAS?$AAi?$AAz?$AAe?$AA?$AA@ 100010f4     FARCmds.obj
 0001:0000010c       ??_C@_1BK@LOJIPNKK@?$AAE?$AAd?$AAi?$AAt?$AAN?$AAe?$AAw?$AAF?$AAi?$AAl?$AAe?$AAs?$AA?$AA@ 1000110c     FARCmds.obj
 0001:00000128       ??_C@_1BM@BMDAMABJ@?$AAV?$AAi?$AAe?$AAw?$AAZ?$AAe?$AAr?$AAo?$AAF?$AAi?$AAl?$AAe?$AAs?$AA?$AA@ 10001128     FARCmds.obj
 0001:00000144       ??_C@_1BE@EKEFMMPP@?$AAC?$AAa?$AAt?$AAc?$AAh?$AAM?$AAo?$AAd?$AAe?$AA?$AA@ 10001144     FARCmds.obj
 0001:00000158       ??_C@_1BM@IEHCKIMD@?$AAS?$AAh?$AAo?$AAw?$AAC?$AAm?$AAd?$AAO?$AAu?$AAt?$AAp?$AAu?$AAt?$AA?$AA@ 10001158     FARCmds.obj
 0001:00000174       _MainGuid                  10001174     FARCmds.obj
 0001:00000184       _ConfigMenuGuid            10001184     FARCmds.obj
 0001:00000194       _DialogGuid                10001194     FARCmds.obj
 0001:000001a4       ??_C@_1DE@BGKMIKPD@?$AAE?$AAu?$AAg?$AAe?$AAn?$AAe?$AA?5?$AAR?$AAo?$AAs?$AAh?$AAa?$AAl?$AA?5?$AA?$CG?$AA?5?$AAF?$AAa?$AAr?$AA?5?$AAG?$AAr?$AAo?$AAu?$AAp?$AA?$AA@ 100011a4     FARCmds.obj
 0001:000001d8       ??_C@_1EI@IHKPBHMH@?$AAF?$AAA?$AAR?$AA?5?$AAC?$AAo?$AAm?$AAm?$AAa?$AAn?$AAd?$AAs?$AA?5?$AAP?$AAl?$AAu?$AAg?$AAi?$AAn?$AA?5?$AAf?$AAo?$AAr?$AA?5?$AAF?$AAa?$AAr?$AA?5?$AAM?$AAa?$AAn?$AAa@ 100011d8     FARCmds.obj
 0001:00000220       ??_C@_1BA@LGNBLCFH@?$AAF?$AAA?$AAR?$AAC?$AAm?$AAd?$AAs?$AA?$AA@ 10001220     FARCmds.obj
 0001:00000230       ??_C@_13HOIJIPNN@?$AA?5?$AA?$AA@ 10001230     FARCmds.obj
 0001:00000238       ??_C@_1GC@PBJAIBOO@?$AAv?$AAi?$AAe?$AAw?$AA?3?$AAe?$AAd?$AAi?$AAt?$AA?3?$AAg?$AAo?$AAt?$AAo?$AA?3?$AAc?$AAl?$AAi?$AAp?$AA?3?$AAw?$AAh?$AAe?$AAr?$AAe?$AAi?$AAs?$AA?3?$AAl?$AAi?$AAn?$AAk@ 10001238     FARCmds.obj
 0001:0000029c       ??_7?$DialogItemBinding@UFarDialogItem@@@@6B@ 1000129c     FARCmds.obj
 0001:000002a4       ??_7?$DialogBuilderBase@UFarDialogItem@@@@6B@ 100012a4     FARCmds.obj
 0001:000002c8       ??_C@_15EFLNJKHH@?$AA?$CF?$AAu?$AA?$AA@ 100012c8     FARCmds.obj
 0001:000002d0       ??_7PluginUIntEditFieldBinding@@6B@ 100012d0     FARCmds.obj
 0001:000002d8       ??_7PluginDialogBuilder@@6B@ 100012d8     FARCmds.obj
 0001:000002fc       ??_7PluginCheckBoxBinding@@6B@ 100012fc     FARCmds.obj
 0001:00000304       ??_7PluginRadioButtonBinding@@6B@ 10001304     FARCmds.obj
 0001:0000030c       ??_7PluginIntEditFieldBinding@@6B@ 1000130c     FARCmds.obj
 0001:00000314       ??_C@_11LOCGONAA@?$AA?$AA@ 10001314     FARCmds.obj
 0001:00000318       ??_C@_1O@BJPKKLLM@?$AAC?$AAo?$AAn?$AAf?$AAi?$AAg?$AA?$AA@ 10001318     FARCmds.obj
 0001:00000328       ??_C@_15BNIPFGCG@?$AA$?$AA?$CK?$AA?$AA@ 10001328     Mix.obj
 0001:00000330       ??_C@_1BE@EKCMLKPN@?$AA?$CF?$AAC?$AAO?$AAM?$AAS?$AAP?$AAE?$AAC?$AA?$CF?$AA?$AA@ 10001330     Mix.obj
 0001:00000344       ??_C@_0BC@KFCLBIA@?$AB?$BE?$AC?$AA?$AA?$AA?$AA?$AA?$MA?$AA?$AA?$AA?$AA?$AA?$AAF?$JL?$AA@ 10001344     Mix.obj
 0001:00000358       ??_C@_13FPGAJAPJ@?$AA?2?$AA?$AA@ 10001358     OpenCmd.obj
 0001:0000035c       ??_C@_1BE@BNONMOPA@?$AA?2?$AA?2?$AA?4?$AA?2?$AAc?$AAd?$AAr?$AAo?$AAm?$AA?$AA@ 1000135c     OpenCmd.obj
 0001:00000370       ??_C@_1CE@JKDBMIKG@?$AA?2?$AA?2?$AA?4?$AA?2?$AAP?$AAh?$AAy?$AAs?$AAi?$AAc?$AAa?$AAl?$AAD?$AAr?$AAi?$AAv?$AAe?$AA?$AA@ 10001370     OpenCmd.obj
 0001:00000394       ??_C@_19BKJMDJK@?$AA?2?$AA?2?$AA?4?$AA?2?$AA?$AA@ 10001394     OpenCmd.obj
 0001:000003a0       ??_C@_17IJMNDCL@?$AA?$CF?$AAl?$AAu?$AA?$AA@ 100013a0     OpenCmd.obj
 0001:000003a8       ??_C@_1BA@EIPEFBMB@?$AA?$CF?$AAl?$AAu?$AA?1?$AA?$CF?$AAl?$AAu?$AA?$AA@ 100013a8     OpenCmd.obj
 0001:000003c0       ??_C@_1GK@PPEHOOAL@?$AAS?$AAO?$AAF?$AAT?$AAW?$AAA?$AAR?$AAE?$AA?2?$AAM?$AAi?$AAc?$AAr?$AAo?$AAs?$AAo?$AAf?$AAt?$AA?2?$AAW?$AAi?$AAn?$AAd?$AAo?$AAw?$AAs?$AA?2?$AAC?$AAu?$AAr?$AAr?$AAe@ 100013c0     OpenCmd.obj
 0001:0000042c       ??_C@_13PJJBFPED@?$AA?$DL?$AA?$AA@ 1000142c     OpenCmd.obj
 0001:00000430       ??_C@_1BA@HAHEJCII@?$AAP?$AAA?$AAT?$AAH?$AAE?$AAX?$AAT?$AA?$AA@ 10001430     OpenCmd.obj
 0001:00000440       ??_C@_19IJOJOJIB@?$AAP?$AAA?$AAT?$AAH?$AA?$AA@ 10001440     OpenCmd.obj
 0001:0000044c       ??_C@_1BA@IBNPAI@?$AAF?$AAA?$AAR?$AAH?$AAO?$AAM?$AAE?$AA?$AA@ 1000144c     OpenCmd.obj
 0001:0000045c       ??_C@_15GBHPEJPD@?$AA?1?$AAS?$AA?$AA@ 1000145c     OpenCmd.obj
 0001:00000464       ??_C@_15MDAMMGLB@?$AA?1?$AAN?$AA?$AA@ 10001464     OpenCmd.obj
 0001:0000046c       ??_C@_19JMGCACDF@?$AA?1?$AAM?$AAS?$AAG?$AA?$AA@ 1000146c     OpenCmd.obj
 0001:00000478       ??_C@_13NEIAEHFG@?$AA?$CC?$AA?$AA@ 10001478     OpenCmd.obj
 0001:0000047c       ??_C@_1BM@MDBPDFDA@?$AA?$CF?$AAC?$AAO?$AAM?$AAS?$AAP?$AAE?$AAC?$AA?$CF?$AA?5?$AA?1?$AAc?$AA?5?$AA?$AA@ 1000147c     OpenCmd.obj
 0001:00000498       ??_C@_1BC@ENICKDH@?$AAC?$AAo?$AAn?$AAt?$AAe?$AAn?$AAt?$AAs?$AA?$AA@ 10001498     OpenCmd.obj
 0001:000004ac       ??_C@_17KKFGGCGH@?$AAR?$AAU?$AAN?$AA?$AA@ 100014ac     OpenCmd.obj
 0001:000004b4       ??_C@_17NMIMIGP@?$AAR?$AAu?$AAn?$AA?$AA@ 100014b4     OpenCmd.obj
 0001:000004bc       ??_C@_19JHOCBEIE@?$AAV?$AAI?$AAE?$AAW?$AA?$AA@ 100014bc     OpenCmd.obj
 0001:000004c8       ??_C@_19MJAKNMNK@?$AAV?$AAi?$AAe?$AAw?$AA?$AA@ 100014c8     OpenCmd.obj
 0001:000004d4       ??_C@_19PEJAKIIO@?$AAC?$AAL?$AAI?$AAP?$AA?$AA@ 100014d4     OpenCmd.obj
 0001:000004e0       ??_C@_19KKHIGANA@?$AAC?$AAl?$AAi?$AAp?$AA?$AA@ 100014e0     OpenCmd.obj
 0001:000004ec       ??_C@_1BA@NBLHMMII@?$AAW?$AAH?$AAE?$AAR?$AAE?$AAI?$AAS?$AA?$AA@ 100014ec     OpenCmd.obj
 0001:000004fc       ??_C@_1BA@BCPLKBBA@?$AAW?$AAh?$AAe?$AAr?$AAe?$AAI?$AAs?$AA?$AA@ 100014fc     OpenCmd.obj
 0001:0000050c       ??_C@_19KFAJFECL@?$AAE?$AAD?$AAI?$AAT?$AA?$AA@ 1000150c     OpenCmd.obj
 0001:00000518       ??_C@_19PLOBJMHF@?$AAE?$AAd?$AAi?$AAt?$AA?$AA@ 10001518     OpenCmd.obj
 0001:00000524       ??_C@_19MEMGFJJL@?$AAG?$AAO?$AAT?$AAO?$AA?$AA@ 10001524     OpenCmd.obj
 0001:00000530       ??_C@_19JKCOJBMF@?$AAG?$AAo?$AAt?$AAo?$AA?$AA@ 10001530     OpenCmd.obj
 0001:0000053c       ??_C@_19NHGGBNEB@?$AAL?$AAI?$AAN?$AAK?$AA?$AA@ 1000153c     OpenCmd.obj
 0001:00000548       ??_C@_19IJIONFBP@?$AAL?$AAi?$AAn?$AAk?$AA?$AA@ 10001548     OpenCmd.obj
 0001:00000554       ??_C@_19LIDMLGEF@?$AAL?$AAO?$AAA?$AAD?$AA?$AA@ 10001554     OpenCmd.obj
 0001:00000560       ??_C@_19OGNEHOBL@?$AAL?$AAo?$AAa?$AAd?$AA?$AA@ 10001560     OpenCmd.obj
 0001:0000056c       ??_C@_1O@PAPHGGOK@?$AAU?$AAN?$AAL?$AAO?$AAA?$AAD?$AA?$AA@ 1000156c     OpenCmd.obj
 0001:0000057c       ??_C@_1O@PJHDHGJM@?$AAU?$AAn?$AAl?$AAo?$AAa?$AAd?$AA?$AA@ 1000157c     OpenCmd.obj
 0001:0000058c       _IID_IShellLinkW           1000158c     shell32:shguid.obj
 0001:0000059c       _IID_IPersistFile          1000159c     uuid:objidl_i.obj
 0001:000005ac       _CLSID_ShellLink           100015ac     uuid:shguids2.obj
 0001:000005c0       __alloca_probe             100015c0     chkstk.obj
 0001:000005c0       __chkstk                   100015c0 f   chkstk.obj
 0001:000005f0       ?GetLangString@PluginDialogBuilder@@MAEPB_WH@Z 100015f0 f i FARCmds.obj
 0001:00000610       _GetGlobalInfoW@4          10001610 f   FARCmds.obj
 0001:00000690       _SetStartupInfoW@4         10001690 f   FARCmds.obj
 0001:000008f0       _OpenW@4                   100018f0 f   FARCmds.obj
 0001:00000b80       _GetPluginInfoW@4          10001b80 f   FARCmds.obj
 0001:00000bd0       ?SaveValue@?$DialogItemBinding@UFarDialogItem@@@@UAEXPAUFarDialogItem@@H@Z 10001bd0 f i FARCmds.obj
 0001:00000bd0       ?InitDialogItem@?$DialogBuilderBase@UFarDialogItem@@@@MAEXPAUFarDialogItem@@PB_W@Z 10001bd0 f i FARCmds.obj
 0001:00000be0       ?TextWidth@?$DialogBuilderBase@UFarDialogItem@@@@MAEHABUFarDialogItem@@@Z 10001be0 f i FARCmds.obj
 0001:00000bf0       ?DoShowDialog@?$DialogBuilderBase@UFarDialogItem@@@@MAEHXZ 10001bf0 f i FARCmds.obj
 0001:00000c00       ?CreateRadioButtonBinding@?$DialogBuilderBase@UFarDialogItem@@@@MAEPAU?$DialogItemBinding@UFarDialogItem@@@@PAH@Z 10001c00 f i FARCmds.obj
 0001:00000c00       ?GetLangString@?$DialogBuilderBase@UFarDialogItem@@@@MAEPB_WH@Z 10001c00 f i FARCmds.obj
 0001:00000c10       ??1?$DialogBuilderBase@UFarDialogItem@@@@MAE@XZ 10001c10 f i FARCmds.obj
 0001:00000c60       ?CreateCheckBoxBinding@?$DialogBuilderBase@UFarDialogItem@@@@MAEPAU?$DialogItemBinding@UFarDialogItem@@@@PAHH@Z 10001c60 f i FARCmds.obj
 0001:00000c60       ?AddUIntEditField@?$DialogBuilderBase@UFarDialogItem@@@@UAEPAUFarDialogItem@@PAIH@Z 10001c60 f i FARCmds.obj
 0001:00000c60       ?AddIntEditField@?$DialogBuilderBase@UFarDialogItem@@@@UAEPAUFarDialogItem@@PAHH@Z 10001c60 f i FARCmds.obj
 0001:00000c70       ??_G?$DialogBuilderBase@UFarDialogItem@@@@MAEPAXI@Z 10001c70 f i FARCmds.obj
 0001:00000c70       ??_E?$DialogBuilderBase@UFarDialogItem@@@@MAEPAXI@Z 10001c70 f i FARCmds.obj
 0001:00000c90       ?ReallocDialogItems@?$DialogBuilderBase@UFarDialogItem@@@@IAEXXZ 10001c90 f i FARCmds.obj
 0001:00000d60       ?UpdateSecondColumnPosition@?$DialogBuilderBase@UFarDialogItem@@@@IAEXXZ 10001d60 f i FARCmds.obj
 0001:00000dc0       ?SaveValues@?$DialogBuilderBase@UFarDialogItem@@@@IAEXXZ 10001dc0 f i FARCmds.obj
 0001:00000e10       ?MaxTextWidth@?$DialogBuilderBase@UFarDialogItem@@@@IAEHXZ 10001e10 f i FARCmds.obj
 0001:00000ed0       ??0PluginUIntEditFieldBinding@@QAE@ABUPluginStartupInfo@@PAPAXHPAIH@Z 10001ed0 f i FARCmds.obj
 0001:00000f70       ?SaveValue@PluginUIntEditFieldBinding@@UAEXPAUFarDialogItem@@H@Z 10001f70 f i FARCmds.obj
 0001:00000fa0       ?InitDialogItem@PluginDialogBuilder@@MAEXPAUFarDialogItem@@PB_W@Z 10001fa0 f i FARCmds.obj
 0001:00000fc0       ?TextWidth@PluginDialogBuilder@@MAEHABUFarDialogItem@@@Z 10001fc0 f i FARCmds.obj
 0001:00000fe0       ?DoShowDialog@PluginDialogBuilder@@MAEHXZ 10001fe0 f i FARCmds.obj
 0001:00001040       ?SaveValue@PluginCheckBoxBinding@@UAEXPAUFarDialogItem@@H@Z 10002040 f i FARCmds.obj
 0001:00001080       ?SaveValue@PluginRadioButtonBinding@@UAEXPAUFarDialogItem@@H@Z 10002080 f i FARCmds.obj
 0001:000010b0       ??0PluginIntEditFieldBinding@@QAE@ABUPluginStartupInfo@@PAPAXHPAHH@Z 100020b0 f i FARCmds.obj
 0001:00001150       ?SaveValue@PluginIntEditFieldBinding@@UAEXPAUFarDialogItem@@H@Z 10002150 f i FARCmds.obj
 0001:00001180       ?CreateCheckBoxBinding@PluginDialogBuilder@@MAEPAU?$DialogItemBinding@UFarDialogItem@@@@PAHH@Z 10002180 f i FARCmds.obj
 0001:000011d0       ?CreateRadioButtonBinding@PluginDialogBuilder@@MAEPAU?$DialogItemBinding@UFarDialogItem@@@@PAH@Z 100021d0 f i FARCmds.obj
 0001:00001220       ??_EPluginDialogBuilder@@UAEPAXI@Z 10002220 f i FARCmds.obj
 0001:00001220       ??_GPluginDialogBuilder@@UAEPAXI@Z 10002220 f i FARCmds.obj
 0001:00001260       ?AddCheckbox@?$DialogBuilderBase@UFarDialogItem@@@@QAEPAUFarDialogItem@@HPAHH_N@Z 10002260 f i FARCmds.obj
 0001:00001390       ?AddRadioButtons@?$DialogBuilderBase@UFarDialogItem@@@@QAEXPAHHQBH_N@Z 10002390 f i FARCmds.obj
 0001:000014f0       ?AddTextBefore@?$DialogBuilderBase@UFarDialogItem@@@@QAEPAUFarDialogItem@@PAU2@H@Z 100024f0 f i FARCmds.obj
 0001:00001620       ?AddSeparator@?$DialogBuilderBase@UFarDialogItem@@@@QAEXPB_W@Z 10002620 f i FARCmds.obj
 0001:00001690       ?AddButtons@?$DialogBuilderBase@UFarDialogItem@@@@QAEXHPBHHH@Z 10002690 f i FARCmds.obj
 0001:000017f0       ?UpdateBorderSize@?$DialogBuilderBase@UFarDialogItem@@@@IAEXXZ 100027f0 f i FARCmds.obj
 0001:000018a0       ??_GPluginUIntEditFieldBinding@@UAEPAXI@Z 100028a0 f i FARCmds.obj
 0001:000018a0       ??_EPluginUIntEditFieldBinding@@UAEPAXI@Z 100028a0 f i FARCmds.obj
 0001:000018a0       ??_GPluginCheckBoxBinding@@UAEPAXI@Z 100028a0 f i FARCmds.obj
 0001:000018a0       ??_E?$DialogItemBinding@UFarDialogItem@@@@UAEPAXI@Z 100028a0 f i FARCmds.obj
 0001:000018a0       ??_G?$DialogItemBinding@UFarDialogItem@@@@UAEPAXI@Z 100028a0 f i FARCmds.obj
 0001:000018a0       ??_GPluginIntEditFieldBinding@@UAEPAXI@Z 100028a0 f i FARCmds.obj
 0001:000018a0       ??_EPluginCheckBoxBinding@@UAEPAXI@Z 100028a0 f i FARCmds.obj
 0001:000018a0       ??_GPluginRadioButtonBinding@@UAEPAXI@Z 100028a0 f i FARCmds.obj
 0001:000018a0       ??_EPluginRadioButtonBinding@@UAEPAXI@Z 100028a0 f i FARCmds.obj
 0001:000018a0       ??_EPluginIntEditFieldBinding@@UAEPAXI@Z 100028a0 f i FARCmds.obj
 0001:000018c0       ??0PluginDialogBuilder@@QAE@ABUPluginStartupInfo@@ABU_GUID@@1HPB_WP6GHPAXHH3@Z3_K@Z 100028c0 f i FARCmds.obj
 0001:000019d0       ?AddIntEditField@PluginDialogBuilder@@UAEPAUFarDialogItem@@PAHH@Z 100029d0 f i FARCmds.obj
 0001:00001a90       ?AddUIntEditField@PluginDialogBuilder@@UAEPAUFarDialogItem@@PAIH@Z 10002a90 f i FARCmds.obj
 0001:00001b50       _ConfigureW@4              10002b50 f   FARCmds.obj
 0001:00001ee0       ?GetMsg@@YAPB_WH@Z         10002ee0 f   Mix.obj
 0001:00001f00       ?ExpandEnv@@YAPA_WPB_WPAK@Z 10002f00 f   Mix.obj
 0001:00001f60       ?GetInt@@YAHPB_WPA_W@Z     10002f60 f   Mix.obj
 0001:00002040       ?ReplaceStrings@@YAHPA_WPB_W1HH@Z 10003040 f   Mix.obj
 0001:000021c0       ?PartCmdLine@@YAHPB_WPAPA_W1@Z 100031c0 f   Mix.obj
 0001:00002450       ?ProcessOSAliases@@YAPA_WPB_W@Z 10003450 f   Mix.obj
 0001:00002670       ?GetShellLinkPath@@YAPA_WPB_W@Z 10003670 f   Mix.obj
 0001:000028f0       ?StrToGuid@@YA_NPB_WPAU_GUID@@@Z 100038f0 f   Mix.obj
 0001:00002910       ?IsTextUTF8@@YA_NPBDI@Z    10003910 f   Mix.obj
 0001:00002980       ?GetCPBuffer@@YAIPBXIPAI@Z 10003980 f   Mix.obj
 0001:00002a50       ?ConvertBuffer@@YAPA_WPA_WIHAAIPA_N@Z 10003a50 f   Mix.obj
 0001:00002b70       ??0ConsoleTitle@@QAE@PB_W@Z 10003b70 f i OpenCmd.obj
 0001:00002be0       ??1ConsoleTitle@@QAE@XZ    10003be0 f i OpenCmd.obj
 0001:00002c00       ??0MakeVETitle@@QAE@PB_W0@Z 10003c00 f i OpenCmd.obj
 0001:00002e10       ?isDevice@@YA_NPB_W0@Z     10003e10 f i OpenCmd.obj
 0001:00003160       ?ThreadWhatUpdateScreen@@YGKPAX@Z 10004160 f   OpenCmd.obj
 0001:000037a0       ?__proc_Load@@YAPA_WHPA_W@Z 100047a0 f   OpenCmd.obj
 0001:00003800       ?__proc_Unload@@YAPA_WHPA_W@Z 10004800 f   OpenCmd.obj
 0001:000038f0       ?__proc_Goto@@YAPA_WHPA_W@Z 100048f0 f   OpenCmd.obj
 0001:00003950       ?__proc_WhereIs@@YAPA_WHPA_W_N@Z 10004950 f   OpenCmd.obj
 0001:00003e60       ?__proc_Link@@YA_NHPA_W@Z  10004e60 f   OpenCmd.obj
 0001:00004340       ?OpenFromCommandLine@@YAPA_WPB_W@Z 10005340 f   OpenCmd.obj
 0001:00005120       _memcpy                    10006120 f   libCRT:memcpy.obj
 0001:00005150       _free                      10006150 f   libCRT:free.obj
 0001:00005170       _malloc                    10006170 f   libCRT:malloc.obj
 0001:00005190       ??_V@YAXPAX@Z              10006190 f   libCRT:delete_array.obj
 0001:000051a0       ??_U@YAPAXI@Z              100061a0 f   libCRT:new_array.obj
 0001:000051b0       _memset                    100061b0 f   libCRT:memset.obj
 0001:000051f0       ??3@YAXPAX@Z               100061f0 f   libCRT:delete.obj
 0001:00005200       ??2@YAPAXI@Z               10006200 f   libCRT:new.obj
 0001:00005210       _wcschr                    10006210 f   libCRT:strchr.obj
 0001:00005240       _wcsstr                    10006240 f   libCRT:strstr.obj
 0001:000052a0       _memmove                   100062a0 f   libCRT:memmove.obj
 0001:000052f0       __memicmp                  100062f0 f   libCRT:memicmp.obj
 0001:00005360       _realloc                   10006360 f   libCRT:realloc.obj
 0001:000053b0       _swab                      100063b0 f   libCRT:swab.obj
 0001:000053f4       __IMPORT_DESCRIPTOR_KERNEL32 100063f4     kernel32:KERNEL32.dll
 0001:00005408       __IMPORT_DESCRIPTOR_USER32 10006408     user32:USER32.dll
 0001:0000541c       __IMPORT_DESCRIPTOR_ADVAPI32 1000641c     advapi32:ADVAPI32.dll
 0001:00005430       __IMPORT_DESCRIPTOR_ole32  10006430     ole32:ole32.dll
 0001:00005444       __IMPORT_DESCRIPTOR_RPCRT4 10006444     rpcrt4:RPCRT4.dll
 0001:00005458       __NULL_IMPORT_DESCRIPTOR   10006458     kernel32:KERNEL32.dll
 0002:00000000       ?OptName@@3UOptionsName@@A 10007000     FARCmds.obj
 0002:000000b0       ?Info@@3UPluginStartupInfo@@A 100070b0     FARCmds.obj
 0002:00000138       ?FSF@@3UFarStandardFunctions@@A 10007138     FARCmds.obj
 0002:000001f8       ?Opt@@3UOptions@@A         100071f8     FARCmds.obj

 entry point at        0000:00000000

 Static symbols

 0001:00002350       ?GetAlias@@YAPA_WPB_W0@Z   10003350 f   Mix.obj
 0001:00002c70       ?getCurrDir@@YAPA_W_N@Z    10003c70 f   OpenCmd.obj
 0001:00002cd0       ?closeHandle@@YAXAAPAX@Z   10003cd0 f   OpenCmd.obj
 0001:00002cf0       ?killTemp@@YAXPA_W@Z       10003cf0 f   OpenCmd.obj
 0001:00002d20       ?createFile@@YAPAXPA_WH@Z  10003d20 f   OpenCmd.obj
 0001:00002db0       ?createFileStream@@YAXPB_WPAXPAUTShowOutputStreamData@@1@Z 10003db0 f   OpenCmd.obj
 0001:00002e70       ?validForView@@YA_NPB_W_N1@Z 10003e70 f   OpenCmd.obj
 0001:00003080       ?showPartOfOutput@@YAKPAUTShowOutputStreamData@@_N@Z 10004080 f   OpenCmd.obj
 0001:000032d0       ?MakeTempNames@@YA_NPAPA_W0@Z 100042d0 f   OpenCmd.obj
 0001:00003450       ?loadFile@@YAPA_WPB_WKHAAIAA_N@Z 10004450 f   OpenCmd.obj
 0001:00003600       ?GetStreamAndMode@@YAXAAPA_WAAH1@Z 10004600 f   OpenCmd.obj
 0001:000036b0       ?__getContent@@YAPA_WHPA_W@Z 100046b0 f   OpenCmd.obj
 0001:00004090       ?GetEditParam@@YAPA_WPA_WAAH1AA_N@Z 10005090 f   OpenCmd.obj
 0001:00004180       ?MakeExecuteString@@YAPB_WPB_W@Z 10005180 f   OpenCmd.obj
